S0220000687474703A2F2F737265636F72642E736F75726365666F7267652E6E65742F1D
S12300000C9438000C94CF260C948B1F0C945F000C945F000C945F000C949B1E0C945F00D0
S12300200C945F000C94CE280C945F000C948A2C0C945F000C94A5200C947F200C94E91E88
S12300400C944B2D0C945F000C94702D0C945F000C94052E0C94CD2D0C945F000C945F00DE
S12300600C945F000C945F000C945F000C945F0011241FBECFEFD0E1DEBFCDBF14BEA895C7
S123008088E10FB6F89480936000109260000FBE13E0A0E0B1E0E8EAFFE502C005900D92B0
S12300A0A23FB107D9F718E0A2EFB3E001C01D92A539B107E1F70E9430170C94D22F0C94AF
S12300C000009C01F999FECF32BD21BDF89A80B508959C01F999FECF1FBA32BD21BD60BD30
S12300E00FB6F894FA9AF99A0FBE089520E030E0F999FECF28593D4F32BD21BD28563240E1
S1230100F89A80B5F901E25AF94F80832F5F3F4F81E02034380761F720E030E0F999FECFBC
S123012028573E4F32BD21BD28583140F89A80B5F901E25CFE4F80832F5F3F4F25303105FB
S123014069F712BC11BC089580E090E0FC01E25AF94FE081F999FECF1FBA88599D4F92BDFD
S123016081BDE0BD0FB6F894FA9AF99A0FBE8756924021E08034920749F712BC11BC0895E6
S123018020E030E0F999FECF205F3F4F32BD21BD20513040F89A80B5F901E153FB4F8083EF
S12301A02F5F3F4F81E02034380761F712BC11BC089580E090E0FC01E153FB4FE081F9995D
S12301C0FECF1FBA409692BD81BDE0BD0FB6F894FA9AF99A0FBE0F9721E08034920759F7EC
S12301E012BC11BC089520E430E0F999FECF205B3E4F32BD21BD20553140F89A80B5F901D4
S1230200EB5BFE4F80832F5F3F4F203A310569F712BC11BC089580E490E0FC01EB5BFE4F9C
S1230220E081F999FECF1FBA805B9E4F92BD81BDE0BD0FB6F894FA9AF99A0FBE8F54914036
S1230240803A910551F712BC11BC0895F999FECF82E090E092BD81BDF89A80B590E09093B2
S1230260200180931F0140911F0150912001F999FECF83E090E092BD81BDF89A20B5922F4C
S123028080E0840F951F9093200180931F01F999FECF8DEE93E092BD81BDF89A80B590E02B
S12302A090932401809323014091230150912401F999FECF8EEE93E092BD81BDF89A20B57E
S12302C0922F80E0840F951F909324018093230180911F0190912001909322018093210145
S12302E0F999FECF84E090E092BD81BDF89A80B590E09093260180932501409125015091A8
S12303002601F999FECF85E090E092BD81BDF89A20B5922F80E0840F951F909326018093C5
S12303202501F999FECF86E090E092BD81BDF89A80B590E09093010180930001409100018F
S123034050910101F999FECF87E090E092BD81BDF89A20B5922F80E0840F951F90930101FF
S123036080930001F999FECF81E090E092BD81BDF89A80B58093F203F999FECF88E090E0A2
S123038092BD81BDF89A80B580931301F999FECF89E591E092BD81BDF89A80B580932F0109
S12303A0F999FECF82E094E092BD81BDF89A90B5892F8150883078F080912F01843039F4D5
S12303C081E08093180183E68093140606C082E08093180102C090931801F999FECF89E0DC
S12303E090E092BD81BDF89A80B580931201F999FECF84E094E092BD81BDF89A80B5809371
S1230400BD048091BD04823E14F482EE05C08091BD048F311CF08EE18093BD04F999FECF08
S12304208EE090E092BD81BDF89A80B580932801F999FECF8BE090E092BD81BDF89A80B5BC
S123044020911801829FC001112490931A0180931901F999FECF83E094E092BD81BDF89AF7
S123046080B580931B01F999FECF8CE090E092BD81BDF89A80B520911801829FC0011124A4
S123048090931D0180931C01F999FECF8FE691E092BD81BDF89A80B580931E01F999FECFBD
S12304A082EF91E092BD81BDF89A80B58093670480916704882319F081E080936704F999E3
S12304C0FECF8DE090E092BD81BDF89A80B526E0829FC00111249093150180931401F9990A
S12304E0FECF81E791E092BD81BDF89A80B580933806F999FECF80E791E092BD81BDF89A57
S123050080B5809336068AE08093C70781E08093C507F999FECF8FE891E092BD81BDF89A62
S123052080B5809330018091300181FF05C080913001827F809330018091300185FF05C0A5
S1230540809130018F7280933001F999FECF84EF91E092BD81BDF89A80B590E02CE231E0EA
S1230560AC01429FC001439F900D529F900D11249093CB048093CA04F999FECF85EF91E0CF
S123058092BD81BDF89A80B58093C704F999FECF86EF91E092BD81BDF89A80B58093C504B0
S12305A0F999FECF87EF91E092BD81BDF89A80B58093C404F999FECF88EF91E092BD81BDEE
S12305C0F89A80B590E09093C3048093C2044091C2045091C304F999FECF89EF91E092BD47
S12305E081BDF89A20B5922F80E0840F951F9093C3048093C204F999FECF8BEF91E092BD8E
S123060081BDF89A80B590E090933201809331014091310150913201F999FECF8CEF91E064
S123062092BD81BDF89A20B5922F80E0840F951F9093320180933101F999FECF8DEF91E073
S123064092BD81BDF89A80B590E090933401809333014091330150913401F999FECF8EEF3C
S123066091E092BD81BDF89A20B5922F80E0840F951F9093340180933301F999FECF8FEF2D
S123068091E092BD81BDF89A80B590E090937803809377034091770350917803F999FECFF0
S12306A080E092E092BD81BDF89A20B5922F80E0840F951F9093780380937703F999FECF7E
S12306C08BEC93E092BD81BDF89A80B580937F04F999FECF8CEC93E092BD81BDF89A80B5A4
S12306E090E09093810480938004F999FECF8DEC93E092BD81BDF89A80B580938904F99976
S1230700FECF8EEC93E092BD81BDF89A80B58093790320E030E0F999FECF225A3E4F32BDD1
S123072021BD2E553140F89A80B5F901EB51FE4F8083F999FECF2E583E4F32BD21BD2257DE
S12307403140F89A80B5F901EB5EF94F8083F999FECF24583E4F32BD21BD2C573140F89A14
S123076080B5F901EB5EF94F808B2F5F3F4F2A30310509F0D0CFF999FECF87E092E092BDDF
S123078081BDF89A80B580933901F999FECF83E092E092BD81BDF89A80B580933A0120E02D
S12307A030E094E6F901EC55F84F908BF999FECF245E3D4F32BD21BD2C513240F89A80B51E
S12307C0F901EC55F84F80832F5F3F4F2031310549F720E030E0F999FECF27593E4F32BD42
S12307E021BD29563140F89A80B5F901E65DFE4F80832F5F3F4F2430310569F720E030E0BD
S1230800F999FECF225D3D4F32BD21BD2E523240F89A80B5F901E454FC4F80832F5F3F4F48
S12308202031310569F7F999FECF8DE691E092BD81BDF89A80B580932701F999FECF81EF2C
S123084091E092BD81BDF89A80B580936604F999FECF80EF91E092BD81BDF89A80B58093AC
S12308602E01F999FECF86E092E092BD81BDF89A80B58093290120E030E0F999FECF2A5490
S12308803C4F32BD21BD265B3340F89A80B5F901E151FE4F80832F5F3F4F2031310569F7C2
S12308A0F999FECF87EC93E092BD81BDF89A80B580933C01F999FECF88EC93E092BD81BD78
S12308C0F89A80B580933D01F999FECF84ED93E092BD81BDF89A80B580937204F999FECF7D
S12308E085ED93E092BD81BDF89A80B580937304F999FECF86ED93E092BD81BDF89A80B598
S123090080937404F999FECF87ED93E092BD81BDF89A80B580937504F999FECF88ED93E0DB
S123092092BD81BDF89A80B580937604F999FECF89ED93E092BD81BDF89A80B580937704A8
S1230940F999FECF8AED93E092BD81BDF89A80B580937804F999FECF8BED93E092BD81BD90
S1230960F89A80B580937904F999FECF88EE93E092BD81BDF89A80B590E0909336018093A3
S123098035014091350150913601F999FECF89EE93E092BD81BDF89A20B5922F80E0840F0D
S12309A0951F9093360180933501F999FECF8AEE93E092BD81BDF89A80B580936904F9992C
S12309C0FECF8CEC93E092BD81BDF89A80B52AE0829FC00111249093810480938004F99915
S12309E0FECF81ED93E092BD81BDF89A80B52AE0829FC00111249093860480938504F999F5
S1230A00FECF82ED93E092BD81BDF89A80B52AE0829FC0011124909388048093870412BC93
S1230A2011BC089520911F0130912001F999FECF1FBA82E090E092BD81BD20BD0FB6F894D0
S1230A40FA9AF99A0FBE20911F0130912001F999FECF1FBA83E090E092BD81BD30BD0FB6A1
S1230A60F894FA9AF99A0FBE2091250130912601F999FECF1FBA84E090E092BD81BD20BDBD
S1230A800FB6F894FA9AF99A0FBE2091250130912601F999FECF1FBA85E090E092BD81BDB4
S1230AA030BD0FB6F894FA9AF99A0FBE2091000130910101F999FECF1FBA86E090E092BD2E
S1230AC081BD20BD0FB6F894FA9AF99A0FBE2091000130910101F999FECF1FBA87E090E02E
S1230AE092BD81BD30BD0FB6F894FA9AF99A0FBE20911301F999FECF1FBA88E090E092BD0F
S1230B0081BD20BD0FB6F894FA9AF99A0FBE20911201F999FECF1FBA89E090E092BD81BD0F
S1230B2020BD0FB6F894FA9AF99A0FBE12BC11BC0895F999FECF1FBA81EF91E092BD81BDB1
S1230B4010BC0FB6F894FA9AF99A0FBEF999FECF1FBA80EF91E092BD81BD8AE080BD0FB66F
S1230B60F894FA9AF99A0FBE20916704F999FECF1FBA82EF91E092BD81BD20BD0FB6F89400
S1230B80FA9AF99A0FBEF999FECF1FBA89E591E092BD81BD84E080BD0FB6F894FA9AF99AA0
S1230BA00FBEF999FECF1FBA81E092E092BD81BD87E180BD0FB6F894FA9AF99A0FBEF99950
S1230BC0FECF1FBA82E092E092BD81BD8EE180BD0FB6F894FA9AF99A0FBEF999FECF1FBAE1
S1230BE08CE090E092BD81BD85E080BD0FB6F894FA9AF99A0FBEF999FECF1FBA8FE691E083
S1230C0092BD81BD82E380BD0FB6F894FA9AF99A0FBEF999FECF1FBA81E791E092BD81BDBE
S1230C2084E180BD0FB6F894FA9AF99A0FBEF999FECF1FBA80E791E092BD81BD81E080BD8E
S1230C400FB6F894FA9AF99A0FBEF999FECF1FBA84EF91E092BD81BD88EC80BD0FB6F894A0
S1230C60FA9AF99A0FBEF999FECF1FBA85EF91E092BD81BD81E080BD0FB6F894FA9AF99ABC
S1230C800FBEF999FECF1FBA86EF91E092BD81BD84E180BD0FB6F894FA9AF99A0FBEF9995F
S1230CA0FECF1FBA87EF91E092BD81BD8AE580BD0FB6F894FA9AF99A0FBEF999FECF1FBAED
S1230CC088EF91E092BD81BD88EE80BD0FB6F894FA9AF99A0FBEF999FECF1FBA89EF91E082
S1230CE092BD81BD83E080BD0FB6F894FA9AF99A0FBE2091310130913201F999FECF1FBA6F
S1230D008BEF91E092BD81BD20BD0FB6F894FA9AF99A0FBE2091310130913201F999FECFFF
S1230D201FBA8CEF91E092BD81BD30BD0FB6F894FA9AF99A0FBE2091330130913401F999BE
S1230D40FECF1FBA8DEF91E092BD81BD20BD0FB6F894FA9AF99A0FBE209133013091340172
S1230D60F999FECF1FBA8EEF91E092BD81BD30BD0FB6F894FA9AF99A0FBE2091770330919E
S1230D807803F999FECF1FBA8FEF91E092BD81BD20BD0FB6F894FA9AF99A0FBE20917703D3
S1230DA030917803F999FECF1FBA80E092E092BD81BD30BD0FB6F894FA9AF99A0FBEF99998
S1230DC0FECF1FBA87E092E092BD81BD8CED80BD0FB6F894FA9AF99A0FBEF999FECF1FBAD0
S1230DE083E092E092BD81BD86EE80BD0FB6F894FA9AF99A0FBE8CE192E028ECF999FECF45
S1230E001FBA92BD81BD20BD0FB6F894FA9AF99A0FBE019632E08C32930781F7F999FECF6E
S1230E201FBA8FE891E092BD81BD82E280BD0FB6F894FA9AF99A0FBEF999FECF1FBA86E0DC
S1230E4092E092BD81BD81E080BD0FB6F894FA9AF99A0FBE12BC11BC08958F929F92AF92E1
S1230E60BF92CF92DF92EF92FF920F931F93CF93DF93C0E0D0E035E0832E32E0932E23ED18
S1230E80A22E23E0B22EF999FECF92BC81BCF89A60B5F999FECFB2BCA1BCF89AE0B46E014B
S1230EA0CC0CDD1C2FEF31E0C20ED31EF6012081318170E080E090E040E050E00E94432F9F
S1230EC0FF2400E010E0A80197010E94432F24E630E040E050E00E94952F79018A01C80128
S1230EE0B70124EF31E040E050E00E94432F28EC30E040E050E0E20EF31E041F151FA80139
S1230F0097010E94952FCA01B9012FEF30E040E050E00E94432F25E030E040E050E00E94B1
S1230F20952F82E0220F331F441F551F8A95D1F7CA01B90124E630E040E050E00E94952FF1
S1230F40F601318320832196C732D10509F09BCFC0E0D0E009EC802E03E0902E13EDA12EF3
S1230F6013E0B12EF999FECF92BC81BCF89A60B5F999FECFB2BCA1BCF89AE0B46E01CC0C73
S1230F80DD1C2DE432E0C20ED31EF6012081318170E080E090E040E050E00E94432FFF247F
S1230FA000E010E0A80197010E94432F24E630E040E050E00E94952F79018A01C801B701B2
S1230FC024EF31E040E050E00E94432F28EC30E040E050E0E20EF31E041F151FA801970178
S1230FE00E94952FCA01B9012FEF30E040E050E00E94432F25E030E040E050E00E94952FA5
S1231000A2E0220F331F441F551FAA95D1F7CA01B90124E630E040E050E00E94952FF6019D
S1231020318320832196C732D10509F09BCFC0E0D0E0FAEC8F2EF3E09F2EE3EDAE2EE3E06A
S1231040BE2EF999FECF92BC81BCF89A60B5F999FECFB2BCA1BCF89AE0B46E01CC0CDD1C7F
S12310602BE932E0C20ED31EF6012081318170E080E090E040E050E00E94432FFF2400E0B4
S123108010E0A80197010E94432F24E630E040E050E00E94952F79018A01C801B70124EF9E
S12310A031E040E050E00E94432F28EC30E040E050E0E20EF31E041F151FA80197010E9408
S12310C0952FCA01B9012FEF30E040E050E00E94432F25E030E040E050E00E94952F62E024
S12310E0220F331F441F551F6A95D1F7CA01B90124E630E040E050E00E94952FF6013183CB
S123110020832196C732D10509F09BCFC0E0D0E034E0832E32E0932E23EDA22E23E0B22E94
S1231120F999FECF92BC81BCF89A60B5F999FECFB2BCA1BCF89AE0B46E01CC0CDD1C29EE73
S123114032E0C20ED31EF6012081318170E080E090E040E050E00E94432FFF2400E010E0F7
S1231160A80197010E94432F24E630E040E050E00E94952F79018A01C801B70124EF31E09C
S123118040E050E00E94432F28EC30E040E050E0E20EF31E041F151FA80197010E94952F74
S12311A0CA01B9012FEF30E040E050E00E94432F25E030E040E050E00E94952F82E0220FB6
S12311C0331F441F551F8A95D1F7CA01B90124E630E040E050E00E94952FF6013183208358
S12311E02196C732D10509F09BCFDF91CF911F910F91FF90EF90DF90CF90BF90AF909F9049
S12312008F900895EAE7F0E0108210927C0080E880BF87EE808311B885E090E090930104D8
S12312208093000488E790E09093F5038093F40384E690E0909303048093020490930B0440
S123124080930A0486E490E0909305048093040408950F931F93CF93DF93282F30E0F90122
S1231260EE0FFF1FEE5FFE4F0081118183E0033F180718F0E2E3F0E04AC083E00F3D180769
S123128018F0EAE0F0E043C0A0E0B0E087E290E0289FA001299F500D389F500D1124EA01DB
S12312A0CA0FDB1FCC0FDD1FC150DE4F888199818017910730F5FD013197E40FF51FEE0F01
S12312C0FF1FE150FE4F208131816081718148815981FD01EE0FFF1FEE0FFF1FEA0FFB1F5E
S12312E03596201B310BC901880F991F880F991F641B750B820F931F0E946E2FE60FF71FB4
S123130006C01196A732B10551F6E8ECF0E0CF01DF91CF911F910F9108950F931F93CF939F
S1231320DF93AC01E0E0F0E0EF01CC0FDD1FDE01A95CBC4F8D919C91119748175907C0F5DD
S12313406D917C913197EE0FFF1FDF01A95CBC4F8D919C911197681B790B8D919C91C15B4A
S1231360DC4F28813981E15BFC4F00811181481B590B84E690E0DC014A9FC0014B9F900D92
S12313805A9F900D11240E946E2F201B310B0190F081E02D629FC001639F900D729F900DAA
S12313A0112464E670E00E946E2F6E0F7F1F09C03196EA30F10509F0B7CF60916303709189
S12313C06403CB01DF91CF911F910F9108958091F4039091F503282F205527FF0AC080912B
S12313E01401909115019C01220F331F280F391F1FC02F312CF0209114013091150118C01E
S12314004091140150911501332727FD309588E290E0821B930B9C01249FC001259F900D11
S1231420349F900D11246AE070E00E946E2F9B01C90108950F931F93CF93DF93AC01809141
S12314407A0390917B034817590718F4E0EFF0E057C080919603909197038417950718F443
S1231460E0E0F0E04DC0E1E0F0E0EF01CC0FDD1FDE01A658BC4F8D919C91119748175907D9
S1231480C0F56D917C913197EE0FFF1FDF01A658BC4F8D919C911197681B790B8D919C9177
S12314A0E856FC4F20813181C856DC4F08811981481B590B84E690E0DC014A9FC0014B9FCE
S12314C0900D5A9F900D11240E946E2F201B310B0190F081E02D629FC001639F900D729F69
S12314E0900D112464E670E00E946E2FE61BF70B07C03196EE30F10509F0B7CFEEEFF0E06C
S1231500CF01DF91CF911F910F91089580917E04882359F08CED95E090933801809337011E
S123152010929804109297042AC080917E04882349F08CED95E0909338018093370184E6CC
S123154090E019C080917E04882349F08CED95E090933801809337018AEF90E00CC080916C
S12315607E04882361F08CED95E0909338018093370184EF91E09093980480939704F89477
S123158080916204909163048A5A9A4AC1F080916204909163048555954589F07894809186
S12315A09F079091A00780649093A00780939F0784EF91E090933801809337010AC07894F1
S12315C080919F079091A0078F7B9093A00780939F07F89480916404909165048F3F89F025
S12315E0789480919F079091A00780689093A00780939F0784EF91E0909338018093370166
S12316000AC0789480919F079091A0078F779093A00780939F078091370190913801892B91
S1231620B1F15E9A20919704309198042115310511F45E9A19C08091950490919604029723
S123164098F48BB18295869586958370809581708295880F880F807C9BB19F7B982B9BB9BA
S12316603093960420939504809195049091960401979093960480939504809137019091ED
S123168038010197909338018093370108955E981092980410929704089580919F0790914B
S12316A0A0079F779093A00780939F07809100019091010197FD44C08091F20380FF32C0A2
S12316C02091590430915A0480912101909122018C599F4F8217930720F441E050E060E8AF
S12316E032C02091590430915A04809121019091220149978217930720F441E050E068E090
S123170022C02091590430915A048091210190912201845690408217930790F441E050E08D
S123172064E011C02091590430915A0480912101909122018217930718F440E050E802C093
S123174040E050E060E020919F073091A007CA019927869597958827822B932B9093A00780
S123176080939F0720919F073091A007CA0180709078822B932B9093A00780939F0780912B
S123178000019091010192FF32C02091590430915A0480913101909132018217930738F57A
S12317A02091590430915A04809133019091340128173907E0F4809127012091000430915B
S12317C0010490E08217930794F080919F079091A00794609093A00780939F078091F203DD
S12317E080FF03C0416068600BC0506809C080919F079091A0079B7F9093A00780939F07D2
S1231800209102043091030480913A0190E08217930734F480913A01882311F040616860CD
S123182080917304209104043091050490E08F5B9F4F8217930774F480917304882351F042
S123184040628091590490915A04895B9B40A0F0646012C080917304209104043091050405
S123186090E0C296821793073CF480917304882319F0406271E001C070E0809172042091C1
S12318800A0430910B0490E0C296821793076CF480917204882349F040648091590490916D
S12318A05A04855C994008F06460772321F082E38093550402C010925504309906C040FD4B
S12318C002C057FF09C04170507850937C0440937B0460937D0406C010927C0410927B0478
S12318E010927D0460937E040895809100019091010193FF6EC1339906C0809184048F5FA0
S12319008093840402C01092840480918404853108F454C010927F042091590430915A048B
S123192080917703909178038217930778F480917B0490917C04826090937C0480937B0495
S123194080917D04886080937D0409C080917B0490917C048D7F90937C0480937B04809129
S1231960F20383FF16C08091590490915A04855C994078F080917B0490917C0484609093CF
S12319807C0480937B0480917D04826080937D0409C080917B0490917C048B7F90937C0482
S12319A080937B048091800490918104909383048093820484E3809384048EC0809182042C
S12319C090918304892B09F45CC080918204909183040197909383048093820480917F04E0
S12319E0823099F0833030F4882351F0813009F073C019C08330A9F1843009F06DC031C017
S1231A00109283041092820467C080917B0490917C04846090937C0480937B0480917D046E
S1231A20826080937D042091590430915A0480917703909178038217930768F480917B04B9
S1231A4090917C04826090937C0480937B0480917D04806836C080917B0490917C048D7F1D
S1231A600BC090919D04809179038917F0F080917B0490917C048B7F90937C0480937B0458
S1231A802BC0209191043091920421153105E1F08091590490915A048D5D9540A8F02150C8
S1231AA03040309392042093910480917B0490917C04846090937C0480937B0480917D0435
S1231AC0826080937D0408C01092940410929304109292041092910480917D0481FF07C009
S1231AE08091300180FF03C084E68093C60480917F04853009F06DC090919D048091790359
S1231B00891708F05DC080918904823001F180918904813041F48091CF0790E083709070FC
S1231B20892B69F056C0809189048823A1F48091CF0790E083709070892B09F44AC080918A
S1231B401206909113068739910508F442C08AEF80935504089580918904833069F480919A
S1231B607B0490917C04846090937C0480937B0480917D04846021C080918904843069F422
S1231B8080917B0490917C04846090937C0480937B0480917D04886010C08091890485305A
S1231BA0C1F480917B0490917C04846090937C0480937B0480917D04826080937D0408957D
S1231BC080917B0490917C048B7F90937C0480937B0408959C018091F20384FF19C0C9012B
S1231BE0C2979C01B3E0220F331FBA95E1F7880F991F280F391F2455354F442737FD40955F
S1231C00542F60E579E784E090E00E94B72F20C08091F20385FD02C024E61AC0C901C2970B
S1231C209C01F3E0220F331FFA95E1F7880F991F280F391F2455354F442737FD4095542F74
S1231C4060E579E784E090E00E94B72F2C592695822F0895A89582E50E945A2E83E10E941D
S1231C605A2E8091590490915A04892F0E945A2E8091590490915A040E945A2E80910A04D3
S1231C8090910B040E945A2E8091D0078E5C0E945A2E8091F4039091F5030E945A2E80918E
S1231CA00204909103040E945A2E80910004909101040E945A2E8091FC039091FD030E9490
S1231CC05A2E80916004909161046091180170E00E946E2F862F0E945A2E80915D04909172
S1231CE05E0420915F0434E0969587953A95E1F7807F822B0E945A2E80915D0490915E049D
S1231D000E945A2E20919F073091A00780911006909111068870832B0E945A2E80919F07F0
S1231D209091A0070E945A2E8091CD040E945A2E8091C4070E945A2E8091FA039091FB036E
S1231D400E945A2E8091120690911306969587950E945A2E86B1869586958695817090E098
S1231D6090934C0680934B068091B30490E090934E0680934D0686B18695817090E090939B
S1231D80500680934F0680919B0490919C04909352068093510680917D0490E090935406AC
S1231DA08093530680917B0490917C0490935606809355068091FE039091FF0390935806DF
S1231DC08093570680913C0690913D0690935A068093590680919004E82FF0E0EE0FFF1F3C
S1231DE0E55BF94F208131818295807F832B0E945A2EE0919004F0E0EE0FFF1FE55BF94F9E
S1231E00808191810E945A2E8DEA0E945A2E809190048F5F80939004883010F010929004B8
S1231E2008958F929F92AF92BF92CF92DF92EF92FF920F931F93CF93DF93A89588E10FB6A6
S1231E40F89480936000109260000FBE0E94A32E882311F40C94EC160E94372E90938F042E
S1231E6080938E048236910509F47CC48336910508F04FC08D34910509F44DC38E3491051C
S1231E8028F58433910511F40C94AD168533910578F48832910509F482C68932910509F4CF
S1231EA0A8C68132910511F00C94EC160C94C4168534910509F487C18634910509F42EC279
S1231EC08134910511F00C94EC16C1C08535910509F4E8C58635910570F48235910509F496
S1231EE094C58335910509F4E2C68035910511F00C94EC16E4C48835910509F420C681360F
S1231F00910509F452C08735910511F00C94EC1639C58F36910509F429C680379105E8F4B5
S1231F208636910509F4B6C18736910548F48436910509F41DC48536910508F06DC315C4C8
S1231F408936910509F46FC48D36910509F4A2C28736910509F040C78CC48A37910509F447
S1231F605FC48B37910568F48837910509F458C48937910508F067C68037910509F02CC764
S1231F80C5C4863F910509F426C2873F910528F4853F910509F020C79FC1873F910569F1AC
S1231FA0883F910509F018C7AFC081E60E945A2E80EA0E945A2E10928F0410928E040EC01D
S1231FC0E25AF94F80810E945A2E80918E0490918F04019690938F0480938E04E0918E0402
S1231FE0F0918F04E03AF10558F38FEF99E50197F1F7000000C08EE927C087EF0E945A2E34
S123200080EA0E945A2E10928F0410928E040EC0E250F94F80810E945A2E80918E04909188
S12320208F04019690938F0480938E04E0918E04F0918F04E03AF10558F38FEF99E5019711
S1232040F1F7000000C088E00E945A2EC5C610928F0410928E0400E010E0AFEFEA2EA3EB3A
S1232060FA2E0E94A32E882309F446C0C0918E04D0918F04C03AD10579F50E94372E9093D4
S12320808F0480938E048E3B910579F481E40E945A2E81E00E945A2E81E00E945A2E8EEB1A
S12320A00E945A2E06E11AEF27C081E40E945A2E81E00E945A2E80E00E945A2E8EEB0E945C
S12320C05A2EC7010197F1F7000000C0E0918C04F0918D04099510C00E94372EC25AD94FA0
S12320E0888380918E0490918F04019690938F0480938E0400E010E00F5F1F4F2AEF003093
S1232100120708F4AECF68C610928F0410928E04C0E0D0E0FFEFEF2EF3EBFF2E0E94A32EB9
S1232120882309F449C000918E0410918F04003A110579F50E94372E90938F0480938E0473
S12321408730910579F488EF0E945A2E81E00E945A2E81E00E945A2E87E00E945A2EC6E1D2
S1232160DAEF2AC088EF0E945A2E81E00E945A2E80E00E945A2E87E00E945A2EC701019701
S1232180F1F7000000C0E0918C04F0918D04099513C000561F4F0E94372E025A194FF80187
S12321A0808380918E0490918F04019690938F0480938E04C0E0D0E02196FAEFC030DF0709
S12321C008F4ACCF09C6C0E0D0E0E8E1FE2E0AEF10E00E94A32E882309F455C00E94372E50
S12321E08A3B910509F0F8C50FB6F894F0926000109260000FBE10928F0410928E043BC064
S1232200885B0E945A2E8DEF0E945A2E80918E0490918F04809FE001819FD00D909FD00DA7
S1232220112409C0F999FECFD2BDC1BDF89A80B50E945A2E219620918E0430918F042F5F63
S12322403F4F209FC001219F900D309F900D112421503040C817D90728F3822F885B80950A
S12322600E945A2E80918E0490918F04019690938F0480938E0480918E0490918F048430DC
S1232280910508F4BDCF21962AEFC030D20708F4A0CFA2C586E60E945A2E80EA0E945A2E87
S12322A010928F0410928E040EC0E153FB4F80810E945A2E80918E0490918F040196909329
S12322C08F0480938E04E0918E04F0918F04E03AF10558F389E9B8CE85EF0E945A2E80EA50
S12322E00E945A2E10928F0410928E040EC0E159FA4F80810E945A2E80918E0490918F0474
S1232300019690938F0480938E04E0918E04F0918F04E03AF10558F38AE096CE10928F0452
S123232010928E0400E010E07FEFE72E73EBF72E0E94A32E882309F446C0C0918E04D0912A
S12323408F04C03AD10579F50E94372E90938F0480938E04893B910579F486E40E945A2EEB
S123236081E00E945A2E81E00E945A2E89EB0E945A2E06E11AEF27C086E40E945A2E81E0D9
S12323800E945A2E80E00E945A2E89EB0E945A2EC7010197F1F7000000C0E0918C04F0915D
S12323A08D04099510C00E94372EC153DB4F888380918E0490918F04019690938F04809313
S12323C08E0400E010E00F5F1F4F3AEF0030130708F4AECF01C510928F0410928E04C0E000
S12323E0D0E06FEFE62E63EBF62E0E94A32E882309F449C000918E0410918F04003A11057A
S123240079F50E94372E90938F0480938E048930910579F486EF0E945A2E81E00E945A2E02
S123242081E00E945A2E89E00E945A2EC6E1DAEF2AC086EF0E945A2E81E00E945A2E80E096
S12324400E945A2E89E00E945A2EC7010197F1F7000000C0E0918C04F0918D04099513C02F
S123246000561F4F0E94372E01531B4FF801808380918E0490918F04019690938F0480931C
S12324808E04C0E0D0E02196FAEFC030DF0708F4ACCFA2C48DE60E945A2E89E00E945A2ED3
S12324A080911F01909120010E945A2E80911F0190912001892F0E945A2E809125019091CE
S12324C026010E945A2E8091250190912601892F0E945A2E80910001909101010E945A2EE7
S12324E08091000190910101892F0E945A2E809113010E945A2E809112010E945A2EF99992
S1232500FECF89E591E092BD81BDF89A80B50E945A2E82E999CD10928F0410928E04AA2485
S1232520BB245AE0852E912C0E94A32E8A3008F469C00E94372E9093200180931F010091AD
S12325401F01109120010E94372ED82ECC240C0D1D1D1093200100931F010E94372E9093A4
S123256026018093250100912501109126010E94372EF82EEE240E0D1F1D10932601009385
S123258025010E94372E909301018093000100910001109101010E94372ED82FC0E00C0FD3
S12325A01D1F10930101009300010E94372E809313010E94372E809312010E94372EF999AE
S12325C0FECF1FBA92BC81BC80BD0FB6F894FA9AF99A0FBE0E94A3280E94372E823B91057D
S12325E061F40E941205E0918C04F0918D0409954FE6A42E4AEFB42E05C0E0918C04F091AF
S12326008D0409950894A11CB11C20E0A2162AEFB20608F489CFE0C385E60E945A2E83E1E8
S12326200E945A2E10928F0410928E040EC0EB51FE4F80810E945A2E80918E0490918F042A
S1232640019690938F0480938E04E0918E04F0918F04EA30F10558F38091190190911A01AB
S12326606091180170E00E946E2F862F0E945A2E80911C0190911D016091180170E00E9475
S12326806E2F862F0E945A2E8FEF95E30197F1F7000000C080912A010E945A2E80912B01E1
S12326A00E945A2E80912C010E945A2E80912D010E945A2E809114019091150166E070E028
S12326C00E946E2F862F0E945A2E809127010E945A2EF999FECF8EE691E092BD81BDF89A12
S12326E080B50E945A2E8AE90E945A2E8CE60E945A2E84E10E945A2E10928F0410928E0446
S12327000EC0EB5EF94F80810E945A2E80918E0490918F04019690938F0480938E04E09171
S12327208E04F0918F04EA30F10558F310928F0410928E040EC0EB5EF94F80890E945A2E99
S123274080918E0490918F04019690938F0480938E04E0918E04F0918F04EA30F10558F3BA
S123276083E972CC0E94A40037C30E94D90034C381E50E945A2E80E10E945A2E8091B80312
S12327809091B9030E945A2E8091D4079091D5070E945A2E8091D6079091D7070E945A2E04
S12327A08091D8079091D9070E945A2E8091DA079091DB070E945A2E8091DC079091DD07E2
S12327C00E945A2E8091DE079091DF070E945A2E8091FC039091FD030E945A2E80917D04B7
S12327E00E945A2E80917B0490917C040E945A2E8091EA0780950E945A2E80919D040E94BB
S12328005A2E809135060E945A2E84E00E945A2E85E00E945A2E86E00E945A2E8EEA14CCB1
S12328200E942A0ED9C20E94A32E8530E0F30E94372EC82FD0E00E94372EC817D90709F0B7
S1232840CBC20E94372E8C0190938F0480938E040E94372E0817190709F0BEC20E94372E32
S12328608639910509F0B8C280918E04C25AD94F4BC00E94A32E8530E0F30E94372EC82FA1
S1232880D0E00E94372EC817D90709F0A5C20E94372E8C0190938F0480938E040E94372E68
S12328A00817190709F098C20E94372E8839910509F092C280918E04C153DB4F25C00E946F
S12328C0A32E8530E0F30E94372EC82FD0E00E94372EC817D90709F07FC20E94372E8C0159
S12328E090938F0480938E040E94372E0817190709F072C20E94372E8F3A910509F06CC279
S123290080918E04CB5BDE4F888366C2C0E0D0E00E94A32E823080F10E94372E0E94372E96
S12329208F38910509F058C210928F0410928E041CC0EB5BFE4F108180E70E945A2E82E0C7
S12329400E945A2E80918E040E945A2E812F0E945A2E8FE80E945A2E80918E0490918F04AA
S1232960019690938F0480938E04E0918E04F0918F04E03AF105E8F221963AEFC030D307B6
S123298039F62AC20E94A32E8530E0F30E94372EE82ED92E0E94372EF82E0E94372E8C0138
S12329A090938F0480938E040E94372E0817190709F012C28E2D9D2DDF2DC0E08E01080FCE
S12329C0191F0E94372E883A9105C9F4C80161E670E00E94182FBC01607080918E04909105
S12329E08F04682B792B70938F0460938E04C80149E650E00E942E2F12BC11BCEDC1E0910D
S1232A008C04F0918D040995BDCFAA24BB240E94A32E833008F43CC00E94372E082F992E16
S1232A200E94372E182F0E94372E8D3A910509F0D3C1F999FECF802F992DD12ECC24E601A9
S1232A40C80FD91FD2BDC1BDF89A90B5F999FECF2196D2BDC1BD2197F89A80B5F82EEE24E5
S1232A608701090F111D84E50E945A2E84E00E945A2E802F0E945A2E8C2F0E945A2E8D2FE9
S1232A800E945A2E812F0E945A2E8BEA0E945A2E0894A11CB11C80E0A8168AEFB80609F01B
S1232AA0B6CF9AC1AA24BB240E94A32E833008F43CC00E94372E082F992E0E94372E182F14
S1232AC00E94372E8A3A910509F086C1F999FECF802F992DD12ECC24E601C80FD91FD2BD49
S1232AE0C1BDF89A90B5F999FECF2196D2BDC1BD2197F89A80B5F82EEE248701090F111DD5
S1232B0085E50E945A2E84E00E945A2E802F0E945A2E812F0E945A2E8C2F0E945A2E8D2F3B
S1232B200E945A2E8AEA0E945A2E0894A11CB11CE0E0AE16EAEFBE0609F0B6CF4DC1C0E056
S1232B40D0E00E94A32E882359F00E94372E873A910509F041C1E0918C04F0918D04099550
S1232B602196FAEFC030DF0761F736C1C0E0D0E00E94A32E882369F00E94372E803991056F
S1232B8009F02AC10E940B01E0918C04F0918D04099521962AEFC030D20751F71DC1C0E08F
S1232BA0D0E00DE611E00E94A32E8823E1F00E94372E873D910509F00FC18091000490912E
S1232BC00104F999FECF1FBA12BD01BD80BD0FB6F894FA9AF99A0FBE12BC11BCE0918C0409
S1232BE0F0918D04099521963AEFC030D307D9F6F3C0C0E0D0E00EE611E00E94A32E8823A2
S1232C00E1F00E94372E863D910509F0E5C08091000490910104F999FECF1FBA12BD01BDE1
S1232C2080BD0FB6F894FA9AF99A0FBE12BC11BCE0918C04F0918D04099521968AEFC030A2
S1232C40D807D9F6C9C0C0E0D0E00E94A32E823040F10E94372E892B09F0BEC00E94372E5A
S1232C6086389105F1F489E70E945A2E87E00E945A2E8FEC0E945A2E8FE30E945A2E88E043
S1232C800E945A2E83EA0E945A2E85ED0E945A2E84E10E945A2E80E10E945A2E86E80E94A9
S1232CA05A2E2196EAEFC030DE0779F695C0C0E0D0E00E94A32E823008F448C00E94372EDF
S1232CC0892B09F043C00E94372E8C3A910509F083C083E50E945A2E88E00E945A2E80916C
S1232CE06204909163040E945A2E8091620490916304892F0E945A2E80915B0690915C06E2
S1232D000E945A2E80915B0690915C06892F0E945A2E8091390690913A060E945A2E8091C2
S1232D20390690913A06892F0E945A2E8091F0079091F1070E945A2E8091F0079091F107A1
S1232D40892F0E945A2E8CEA0E945A2E2196FAEFC030DF0709F0ADCF3FC0C0E0D0E00E9411
S1232D60A32E823058F00E94372E892BA9F50E94372E8B3C910511F40E94260121962AEF29
S1232D80C030D20761F728C0C0E0D0E004E610E00E94A32E8330D8F00E94372E0197E1F49A
S1232DA00E94372EFC01E09FC001E19F900DF09F900D112490938B0480938A040E94372EF3
S1232DC08E3D910521F010928B0410928A042196FAEFC030DF07E1F6A895DF91CF911F9112
S1232DE00F91FF90EF90DF90CF90BF90AF909F908F900895CF93DF93CFEFD3E222C0CE01E2
S1232E000197F1F7000000C00E94110F2D982C9ACE010197F1F7000000C081E20E945A2E85
S1232E2080E00E945A2E8EED0E945A2E2D9A2C9880918A0490918B04019790938B04809328
S1232E408A0480918A0490918B040B97C0F62D9A2C9A10928B0410928A04DF91CF910895DE
S1232E602F923F924F925F926F927F928F929F92AF92BF92CF92DF92EF92FF920F931F93BC
S1232E80CF93DF9314BEA89588E10FB6F89480936000109260000FBE1092A00710929F07BE
S1232EA00E94A52D259A249A209A219A2D9A2C9A289A299A579A5F9A0000000000000000AC
S1232EC081E08093CC048093C8078093CE0480935D06549A559A5C9A5D9A229A239A569A3A
S1232EE02A9A2B985E980000000052983A983B98439A3A98429A3998419A3898409A0E943F
S1232F00AC2DF999FECF8AE591E092BD81BDF89A80B5809368040E94331E0E94A3280E94C0
S1232F20952D10927A0010927C0080E880BF87EE80937A0011B885E090E09093010480930F
S1232F40000488E790E09093F5038093F40384E690E0909303048093020490930B04809303
S1232F600A0486E490E090930504809304040E942D072A9A2B98F999FECF87E090E092BD3C
S1232F8081BDF89A80B512BC11BC85FFEEC080910001909101019F7D9093010180930001D1
S1232FA00E9412050E9499050E94D9000E94A4000E940B01F999FECF1FBA8AE090E092BD44
S1232FC081BD86E080BD0FB6F894FA9AF99A0FBEF999FECF1FBA8BE090E092BD81BD89E1BD
S1232FE080BD0FB6F894FA9AF99A0FBEF999FECF1FBA8CE090E092BD81BD8EE180BD0FB639
S1233000F894FA9AF99A0FBEF999FECF1FBA8EE090E092BD81BD8EE180BD0FB6F894FA9AF8
S1233020F99A0FBE80E090E0FC01EB51FE4FE081F999FECF1FBA825A9E4F92BD81BDE0BD4A
S12330400FB6F894FA9AF99A0FBE8D5591408A30910551F780E090E0FC01E65DFE4FE0811E
S1233060F999FECF1FBA87599E4F92BD81BDE0BD0FB6F894FA9AF99A0FBE88569140843075
S1233080910551F780E090E0FC01EB5EF94FE081F999FECF1FBA8E589E4F92BD81BDE0BD5A
S12330A00FB6F894FA9AF99A0FBE815791408A30910551F780E090E0FC01EB5EF94F20897F
S12330C0F999FECF1FBA84589E4F92BD81BD20BD0FB6F894FA9AF99A0FBE8B5791408A30CF
S12330E0910551F720913806F999FECF1FBA81E791E092BD81BD20BD0FB6F894FA9AF99A0C
S12331000FBE2091140130911501F999FECF1FBA8DE090E092BD81BDC90166E070E00E949D
S12331206E2F60BD0FB6F894FA9AF99A0FBEF999FECF1FBA8DE691E092BD81BD84E180BD41
S12331400FB6F894FA9AF99A0FBEF999FECF1FBA8EE691E092BD81BD81EE80BD0FB6F8947F
S1233160FA9AF99A0FBE12BC11BC0E94F3000E94260120E030E0F999FECF205F3F4F32BDF3
S123318021BD20513040F89A80B5F901E153FB4F80832F5F3F4F81E02034380761F712BCF4
S12331A011BC0E947600809100019091010185FD07C080916F008B7F80936F002D9A2C9A0F
S12331C080912901882311F480E801C080E480933B011092F30380911401909115018D5A48
S12331E09D4030F08CEA9DE090931501809314011092560486B3866086BB78948AEA0E94FC
S12332005A2E80E00E945A2E85E50E945A2E86B18695817080936A0480916E0083608093CB
S12332206E002A9AFF24F394F4E0BF2EE6E0AE2E72E4972E65E0862E57E8752E47E0642E9C
S123324033E4532E26E4422E9BE4C92ED12C83E0382E04E4202E14E6E12E2B9AA8958091CA
S1233260590490915A048635910568F180915604882349F580919F079091A0079F7E9093B1
S1233280A00780939F0780916F00856080936F0080916E00836080936E002A9AF092560460
S12332A080919F079091A00780629093A00780939F0780919F079091A00790629093A007EB
S12332C080939F074EC020915604213009F049C08091590490915A048234910508F041C093
S12332E080916F008D7F80936F00809170008C7F8093700080916F008B7F80936F00809190
S12333006E00836080936E0080919F079091A0078F7D9093A00780939F0780919F079091F1
S1233320A007877F9093A00780939F072093CC042093C8072093CE0420935D065C9A5D9ACC
S12333402D9A2C9A289A299A1092560480919F079091A0079F7D9093A00780939F0710929B
S1233360540480915604813001F580916F00826080936F0080917000836080937000B5BCA3
S123338080916E00836080936E0080919F079091A00788609093A00780939F072A9A2B9AD3
S12333A010928B0410928A041FC015BC109254042D9A2C9A289A299A109254041092B3009D
S12333C010926104109260048091430190914401892B51F42A9880918A0490918B0485365C
S12333E0910510F00E94FA168091F303833009F4CDC0843018F4882371F072C0853009F48D
S1233400EAC1853008F425C1863009F49BC1873009F068C221C280915704909158048536F6
S1233420910508F461C2E091F303F0E080917800909179008C7F65E070E00E946E2FEE0F9D
S1233440FF1FEC5CFB4F718360838091F303C82FD0E0E091F303F0E0EE0FFF1FEC50FC4F5A
S123346080819181E091F303F0E0EE0FFF1FEC5CFB4F20813181880F991F880F991F820FCF
S1233480931F880F991F6AE070E00E946E2FCC0FDD1FCC50DC4F79836883109258041092A9
S12334A05704F092F30381E480937C000E94110F0E94E70990931701809316018091430133
S12334C090914401892B51F08091430190914401019790934401809343012A9AA89504C2B4
S12334E080915704909158048536910508F4FCC11092580410925704A8958091F3038130E5
S123350041F580910801909109012091780030917900820F931F96958795909309018093FF
S1233520080183E00E9429099093F7038093F6038091F6039091F70390930B0480930A04A6
S1233540E092C90722E02093F30385E480937C00CBC18091020190910301209178003091D3
S12335607900820F931F969587959093030180930201D092F903C092F803D0920504C0929F
S123358004043092F30320927C00AEC180915704909158048536910508F4A6C1E091F303C6
S12335A0F0E080917800909179009695879596958795EE0FFF1FEC5CFB4F918380838091B1
S12335C0F303C82FD0E0E091F303F0E0EE0FFF1FEC50FC4F80819181E091F303F0E0EE0F2A
S12335E0FF1FEC5CFB4F20813181880F991F880F991F820F931F880F991F6AE070E00E9458
S12336006E2FCB01CC0FDD1FCC50DC4F998388831092580410925704B092F30380913B0178
S123362080937C000E94110FA89580917A048F5F80937A04843010F010927A0480917A0487
S1233640982F91709093C0048695817080933B064BC180915704909158048159914008F4BB
S123366043C180912901882329F1E091F303F0E0809178009091790096958795969587955A
S1233680EE0FFF1FEC5CFB4F91838083A091F303B0E0E091F303F0E0EE0FFF1FEC5CFB4FC7
S12336A080819181AA0FBB1FAC50BC4F11969C938E933EC0E091F303F0E080917800909183
S12336C07900EE0FFF1FEC5CFB4F918380838091F303C82FD0E0E091F303F0E0EE0FFF1FA9
S12336E0EC50FC4F00811181E091F303F0E0EE0FFF1FEC5CFB4F808191810E941A0A9C01D2
S1233700220F331F280F391FC801F3E0880F991FFA95E1F7801B910B820F931F6AE070E02D
S12337200E946E2FCC0FDD1FCC50DC4F7983688310925804109257048092F30370927C00C0
S1233740A895D2C080915704909158048536910508F4CAC0E091F303F0E0809178009091F5
S123376079009695879596958795EE0FFF1FEC5CFB4F91838083A091F303B0E0E091F3035C
S1233780F0E0EE0FFF1FEC50FC4F20813181E091F303F0E0EE0FFF1FEC5CFB4F8081918169
S12337A0820F931F880F991F9695879596958795AA0FBB1FAC50BC4F11969C938E931092B2
S12337C05804109257046092F30350927C000E94110FA89589C08091570490915804893C50
S12337E0910508F481C0E091F303F0E08091780090917900EE0FFF1FEC5CFB4F91838083D4
S1233800A091F303B0E0E091F303F0E0EE0FFF1FEC50FC4F20813181E091F303F0E0EE0F8D
S1233820FF1FEC5CFB4F80819181820F931F96958795AA0FBB1FAC50BC4F11969C938E93A6
S12338401092580410925704A092F30390927C000E94110FA89548C08091570490915804B3
S12338608536910508F440C0E091F303F0E08091780090917900969587959695879590E09F
S1233880EE0FFF1FEC5CFB4F91838083A091F303B0E0E091F303F0E0EE0FFF1FEC50FC4FD0
S12338A020813181E091F303F0E0EE0FFF1FEC5CFB4F80819181820F931F96958795AA0F77
S12338C0BB1FAC50BC4F11969C938E9310925804109257041092F30340927C000E94110F69
S12338E0A89502C0F092F30380915704909158040196909358048093570480915904909151
S12339005A048F55914008F448C08091F60787FF02C0E0E002C0E091F6078091C6078F5F7A
S12339208093C6079091C6078091C7079817B8F11092C6072091020430910304AE2FB0E023
S1233940FD01EC55F84F808190E02817390754F48091C407843634F48091C4079091C5071E
S1233960890F12C02091020430910304AC55B84F8C9190E0281739074CF08091C40782307C
S12339802CF08091C40781508093C4078091C40785362CF0E092C40702C0F092C40780916C
S12339A0590490915A048739910508F46DC080912701209100043091010490E0489682170D
S12339C093070CF461C08091C8049091C90401969093C9048093C8042091C8043091C904EC
S12339E08091CA049091CB042817390708F440C01092C9041092C8042091590430915A046F
S1233A008091C2049091C3040A972817390730F49091C6048091C704890F15C0209159045D
S1233A2030915A048091C2049091C30449968217930758F49091C6048091C504891728F4C5
S1233A408091C60481508093C6049091C6048091C404891718F48091C40408C09091C604DD
S1233A608091C504981720F48091C5048093C6048091590490915A048A58924038F4809110
S1233A80C4048093C60402C01092C6048091F20382FF55C08091590490915A04855F914011
S1233AA008F44DC08091590490915A04805D974008F045C0809127012091000430910104A7
S1233AC090E0049682179307D4F1209100043091010480916D0490E00196821793077CF13C
S1233AE080910A0490910B048F36910544F180916E0490916F04A0917004B09171040196DA
S1233B00A11DB11D80936E0490936F04A0937004B093710480916E0490916F04A0917004DF
S1233B20B091710481549D40A340B04008F1F0926C0480919F079091A007916015C0809105
S1233B4000049091010480936D0410926E0410926F04109270041092710410926C0480913A
S1233B609F079091A0079E7F9093A00780939F070E944D0B0E94750C0E94860A80910001D2
S1233B809091010180FF67C08091300180FF11C08091BC04883C28F08091C6048823C9F0DA
S1233BA016C09091C6048091BC048695891790F010C08091300182FF0DC08091BC04883C3F
S1233BC048F080919F079091A00796FF02C05C9A01C05C988091300184FF16C08091BC04BC
S1233BE0883C28F08091C40718165CF12CC02091C4078091BC04332727FD3095869590E087
S1233C00821793070CF11FC08091300186FF1CC08091BC04883CC0F02091590430915A047C
S1233C2080913501909136018217930760F420910204309103048091690490E082179307BA
S1233C4014F45D9A01C05D988091BC04883C28F01092BC0402C05C9A5D9A8091BC048F5F2E
S1233C608093BC04FACA1092800081EF9FEF909389008093880085EF9FEF90938B0080937F
S1233C808A0080E88093810080EC9AED909385008093840083E090E09093D6038093D503AE
S1233CA08091D5039091D60380688093810010925A041092590480916F00876080936F00B9
S1233CC052983A98259A249A2D9A2C9A289A299AF999FECF82E092E092BD81BDF89A80B50E
S1233CE08093BA03F999FECF81E092E092BD81BDF89A80B58093BB038091BB038E3039F0E3
S1233D008091BB03873119F087E18093BB0380916804813021F480916900836003C0809162
S1233D206900826080936900E89A84E08093680080936D0008951F920F920FB60F9211244D
S1233D402F933F938F939F9386B18695869581702091680490E030E08217930789F181E06E
S1233D608093B3048091D0078230E9F48091640490916504880F991F9093650480936404A5
S1233D808091640490916504816090936504809364048091990490919A04019690939A046F
S1233DA0809399040DC08091990490919A04019790939A04809399041092650410926404F7
S1233DC09F918F913F912F910F900FBE0F901F9018951F920F920FB60F9211248F939F9357
S1233DE08091F7078F5F8093F7078091F707882309F44DC080919F079091A007906190935A
S1233E00A00780939F071092560480919F079091A0079F7D9093A00780939F0780916F00A4
S1233E208B7F80936F0080916F008D7F80936F00809170008C7F8093700080916E00836073
S1233E4080936E002D9A2C9A289A299A80919F079091A0078F7D9093A00780939F078091AC
S1233E609F079091A007877F9093A00780939F0781E08093CC048093C8078093CE04809329
S1233E805D065C9A5D9A10925A041092590410929A041092990478949F918F910F900FBE88
S1233EA00F901F9018958091B304813091F41092B30483E08093D0078091B6039091B703BA
S1233EC09093B9038093B8031092B7031092B6030CC08091D0078F5F8093D0078091D00706
S1233EE0853019F481E08093D0078091990490919A048536910530F084E690E090939A0438
S1233F008093990480918400909185009093F5078093F40708951F920F920FB60F921124FB
S1233F208F939F938091B6039091B70301969093B7038093B6039F918F910F900FBE0F90E9
S1233F401F90189580919F079091A00793FD17C08091D007813011F42D9808958091D00733
S1233F60843011F42C9808958091D007823011F4289808958091D007833009F42998089531
S1233F801F938091B404882309F49BC08091B404813059F42D9A299A8091B6039091B703A9
S1233FA090930308809302080EC08091B404823051F42C9A289A8091B6039091B7039093D4
S1233FC0E9078093E8078091B504882319F41092B40464C08091B504813099F480918A0048
S1233FE090918B004E9690938B0080938A008091B4048C598093B4048091B4048093B504D4
S12340004DC08091B504853611F585B190E2892785B980918A0090918B004E9690938B0095
S123402080938A002091FE073091FF07409100085091010880918A0090918B00A0E0B0E048
S1234040281739074A075B0748F52D9A25C08091B504863619F585B190E1892785B9809107
S12340608A0090918B004E9690938B0080938A002091FE073091FF07409100085091010897
S123408080918A0090918B00A0E0B0E0281739074A075B0718F42C9A1092B5048091390616
S12340A090913A06892B49F18091F207882329F18091390690913A0690938B0080938A00E2
S12340C01CC08091F2078823C1F01091F207113021F01091F207123031F48091F2070E9401
S12340E0A21F1093B4048091F0079091F10790938B0080938A001092F2071F9108951F929B
S12341000F920FB60F9211242F933F934F935F936F937F938F939F93AF93BF93EF93FF93E7
S12341200E94C01F2A9A7894FF91EF91BF91AF919F918F917F916F915F914F913F912F91CA
S12341400F900FBE0F901F9018951F920F920FB60F9211248F939F93F8948091D107882393
S123416009F492C080917B0490917C0497FD8CC08091130180958093EA078091EA0790917A
S123418035068C59891B8093EA0790911406943071F1953040F49230C1F19330D8F4913035
S12341A009F072C00AC0973109F44CC0933609F457C09E3009F068C035C08091EA0780935F
S12341C0B20084E08093B1001092CC049093BF0483E018C08091EA078093B20094E0909310
S12341E0B1001092CE0483E08093BF044BC08091EA078093B2009093B10010925D0690938F
S1234200BF0482E0809314063FC08091EA078093B20084E08093B1001092C8079093BF0403
S123422081E0F0CF81E08093DA038091EA078093B20084E08093B1001092CC0410925D06A3
S123424087E1E0CF81E08093DB038091EA0786BD83E085BD1092C8071092CE048EE0D2CF13
S123426081E08093DA038091EA078093B20084E08093B1001092CC0410925D061092CE040F
S12342801092C8079093140678949F918F910F900FBE0F901F901895EF92FF920F931F9343
S12342A0CF93DF93EC0180916704E7E0F0E0E81BF109EE0FFF1FEC50FC4F0190F081E02D78
S12342C080916604E81BF109F7FF02C0E0E0F0E080912E0126E0829FC00111249C012E9F53
S12342E0C0012F9F900D3E9F900D112464E670E00E94822FCB01603A71050CF08FE980938F
S1234300F3078091F3076AE00E94622F8093CC078091CC0780311CF08FE08093CC0780912A
S1234320590490915A04885E934008F0AAC01092CA078FEF8093F6078091CC0724E1820214
S1234340C001112490935E0480935D048091590490915A0464E670E00E946E2F65506093FC
S1234360EF078091590490915A04845F914060F41092EF07E091EF07FF27E7FDF095E25C82
S1234380FE4F808190E0A9C08091EF078430E1F5E0915D04F0915E04E25AF94F2081E09116
S12343A0EF07FF27E7FDF095E25CFE4F6081E091EF07FF27E7FDF095E25CFE4F808190E016
S12343C09093130680931206E0911206F09113068091590490915A044091EF0730E0220F5A
S12343E0331F261B3109845F91406CE94602A0011124840F951FAC01249FC001259F900DEC
S1234400349F900D11243AC0E091EF07FF27E7FDF095E15CFE4F6081E091EF07FF27E7FD27
S1234420F095E25CFE4F4081E091EF07FF27E7FDF095E25CFE4F808190E090931306809366
S12344401206E0911206F09113068091590490915A042091EF0770E0641B7109845F91408C
S12344604CE9240290011124820F931F9C01629FC001639F900D729F900D112464E670E059
S1234480D1C08091590490915A04875F924250F187EC8093CA078091CA076AE00E94622FE9
S12344A08093F6078091CC072091F60744E18402C0011124332727FD3095820F931F90930C
S12344C05E0480935D04E0915D04F0915E04E25AF94F808190E0880F991F909313068093BA
S12344E01206A8C08091590490915A04885E934062E370E00E946E2F6093CA078091CA0718
S12345006AE00E94622F8093F6078091CC072091F60744E18402C0011124332727FD309594
S1234520820F931F90935E0480935D04E0915D04F0915E04E25AF94F808190E0880F991F42
S123454090931306809312068091F60787FD37C08091F60783319CF5E0915D04F0915E045F
S1234560E15AF94F4081E0915D04F0915E04E25AF94F6081E0911206F09113063091CA0724
S12345808091F60726EF8202C0011124830F911D880F991F50E0461B51099C01249FC001DF
S12345A0259F900D349F900D11246AE070E00E94822FE60FF71FF0931306E09312068091C1
S12345C0CC0787FD37C08091CC078F309CF5E0915D04F0915E04EE58F94F4081E0915D047F
S12345E0F0915E04E25AF94F6081E0911206F09113063091F3078091CC0726EF8202C00153
S12346001124830F911D880F991F50E0461B51099C01249FC001259F900D349F900D1124C0
S12346206AE070E00E94822FE60FF71FF0931306E093120680919F079091A007977F90939F
S1234640A00780939F078091100690911106877F909311068093100680917D04882309F4F4
S123466058C080917D0487FD27C080917D04883088F08091CF0790E083709070892B09F464
S123468048C08091CF0767E00E94622F992309F440C012C080917D048430C0F08091CF0745
S12346A090E083709070892B39F08091CF0767E00E94622F992369F580919F079091A007BC
S12346C098609093A00780939F0723C080917D04823050F08091100690911106886090938A
S12346E011068093100615C080917D04882389F080911206909113068739910550F08091E1
S12347001206909113068C58904090931306809312068091CF078F5F8093CF0740919D04F8
S1234720445645310CF044E12091120630911306809112019091550420583040280F311D96
S1234740291B3109842F4C3E0CF48CEE992787FD9095280F391F30939C0420939B042091C2
S12347609B0430919C048091BD044AE08402C0011124820F931F90939C0480939B048091F4
S123478012012091BD0490E080589F4F240290011124820F931FAC014C9FC0014D9F900D49
S12347A05C9F900D1124A0E0B0E08093FE079093FF07A0930008B09301086091FE07709159
S12347C0FF07809100089091010828E037E040E050E00E94952FC901DA018093FE079093D7
S12347E0FF07A0930008B093010880919B0490919C048D5B92403CF04CEBE42E42E0F42E44
S1234800012D112D15C080919B0490919C04059734F435E0E32EF12C012D112D09C0809195
S12348209B0490919C047C010027F7FC0095102F20915B0430915C042C0F3D1F40E050E091
S1234840C801B7010E94432F28E037E040E050E00E94952FCE01821B930BDF91CF911F9160
S12348600F91FF90EF900895DC018091F6078F302CF02FE030E040E050E00BC08091F607DB
S1234880992787FD909501969C01442737FD4095542FF901E454FC4F608170E080E090E002
S12348A09D0140E050E00E94432F28E037E040E050E00E94952FC90108950F931F93CF9300
S12348C0DF938091CC039091CD039093FD078093FC078091CC039091CD03499708F459C28C
S12348E08091F707882349F088EE9DEF9093D8038093D7031092F70753C080915904909192
S12349005A044091D7035091D803895B9B40C0F0E0915B04F0915C042091CC033091CD039D
S12349208091BA0390E0241B350BAC01429FC001439F900D529F900D112464E170E017C0B9
S1234940E0915B04F0915C042091CC033091CD038091BA0390E0241B350BAC01429FC00185
S1234960439F900D529F900D11246EE170E00E94822FCB018E0F9F1F62E070E00E94822FF3
S123498070935C0460935B0410925C0410925B048091CC039091CD039093D8038093D7039F
S12349A080915404893628F4809154048F5F809354048091590490915A048C5D954050F4FE
S12349C02D9B06C02C9B04C0289B02C0299902C01092B4048091590490915A04C091D7033F
S12349E0D091D803D0935C06C0935B0620915B0630915C060091D5031091D603225E3F4FD8
S1234A0040E050E060E070E489E191E00E94B72FCA01B9012EE130E040E050E00E94432F43
S1234A2020EC30E0A901049F9001059F300D149F300D11242050324040E050E00E94952FDA
S1234A4030935A04209359042091AA043091AB044091A8045091A904C901880F991F820F9D
S1234A60931F840F951F96958795969587959093AB048093AA048091A6049091A70490936E
S1234A80A9048093A8048091A4049091A5049093A7048093A6048091A2049091A3049093F6
S1234AA0A5048093A4048091A0049091A1049093A3048093A20480919E0490919F049093F6
S1234AC0A1048093A0048091590490915A0490939F0480939E048091590490915A048D5D37
S1234AE09540B8F080919D0440919E0450919F042091AA043091AB0490E0821B930B840F7F
S1234B00951F9695879596958795855B80939D040FC084E680939D0480915B0490915C04DD
S1234B2064E070E00E94822F70935C0460935B041092F7078091590490915A048C52914099
S1234B40A0F58091D5039091D603039771F58091D007813051F584E090E09093D603809317
S1234B60D5038091D5039091D6038068809381008091840090918500969587959695879531
S1234B809093850080938400D695C795D695C795D093D803C093D70380915B0690915C06E4
S1234BA096958795969587953AC08091590490915A048F5E9240B8F18091D5039091D60331
S1234BC0049789F58091D007813069F583E090E09093D6038093D5038091D5039091D60324
S1234BE08068809381008091840090918500880F991F880F991F9093850080938400CC0F42
S1234C00DD1FCC0FDD1FD093D803C093D70380915B0690915C06880F991F880F991F90939C
S1234C205C0680935B0680915B0690915C060E944C219093F1078093F00780911006909129
S1234C40110683FF3AC0E091B604F091B704CF0183709070892B99F420915B0630915C061D
S1234C6080915B0690915C066AE070E00E946E2F261B370B3093F1072093F00718C02091F1
S1234C803C0180915B0690915C0668E270E00E946E2F30E0629FC001639F900D729F900DE6
S1234CA011248C599F4F9093F1078093F0073196F093B704E093B60404C01092B7041092CE
S1234CC0B6048091590490915A048A58924038F08091F4039091F5038E3691053CF48CE234
S1234CE091E09093FB078093FA0704C01092FB071092FA078091F0079091F1072091160112
S1234D00309117014091FA075091FB07821B930B841B950B9093E7078093E6078091E60778
S1234D209091E70797FF20C08091E6079091E70720915B0630915C064091F0075091F10707
S1234D40820F931F8417950778F48091F0079091F10720915B0630915C064496821B930BFE
S1234D609093E7078093E607F8948091D007823019F481E08093140680915B0690915C0668
S1234D800E943424909389008093880081E08093D1077894DF91CF911F910F9108951F9208
S1234DA00F920FB60F9211242F933F934F935F936F937F938F939F93AF93BF93EF93FF933B
S1234DC0F89420918400309185008091CC039091CD03969587952817390778F48091590457
S1234DE090915A04815D974040F081E090E09093630480936204789419C078940E945D2463
S1234E000E94531F8091620490916304880F991F909363048093620480916204909163042A
S1234E20816090936304809362045F98809110069091110683FF95C0809184009091850022
S1234E409093CD038093CC03109285001092840078948091620490916304880F991F9093AF
S1234E606304809362045F9A20913C0180915B0690915C0668E270E00E946E2F30E0629F88
S1234E80C001639F900D729F900D11248C599F4F9093F1078093F0078091590490915A04E6
S1234EA08051974208F049C080919F079091A00793FD43C08091F0079091F10790938B0062
S1234EC080938A0020915B0630915C0680915B0690915C069695879596958795281B390BF2
S1234EE030933A06209339068091D007813021F08091D007833031F42C9882E08093B4045E
S1234F0081E00DC08091D007843021F08091D007823039F42D9881E08093B40482E0809385
S1234F20F2078EEB90E090933D0680933C0680919F079091A0079F770FC080915B069091D9
S1234F405C068C509E4F90938B0080938A0080919F079091A00790689093A00780939F07DD
S1234F60DFC080918400909185009093CD038093CC031092850010928400789480916204AE
S1234F8090916304880F991F90936304809362045F9A8091590490915A048051974208F0AB
S1234FA0B5C08091E6079091E70785369105ECF11092B4048091590490915A048C5D954038
S1234FC040F48091F20381FF04C081E08093B50402C01092B5048091E6079091E7079093D5
S1234FE08B0080938A0080918A0090918B0090933A06809339068091D007813021F08091CE
S1235000D007833011F481E009C08091D007843021F08091D007823029F482E08093F20701
S12350201092B40484E090E06CC08091E6079091E7078B5B9F4F7CF11092B40484E690E090
S123504090938B0080938A0090933A06809339068091D007813021F08091D007833011F402
S123506081E009C08091D007843021F08091D007823039F482E08093F2070E94A21F10921B
S1235080B40488E290E090933D0680933C0684E18093D90345C08091F0079091F107909322
S12350A08B0080938A0020915B0630915C068091E6079091E707820F931F90933A068093C9
S12350C039068091D007813021F08091D007833029F481E00E94A21F81E00CC08091D00752
S12350E0843021F08091D007823031F482E00E94A21F82E08093B40484E18093D90384EB73
S123510090E090933D0680933C060AC080915B0690915C068C509E4F90938B0080938A008D
S12351202A9A7894FF91EF91BF91AF919F918F917F916F915F914F913F912F910F900FBECF
S12351400F901F90189521EB30E0F90110821092B6001092B2001092B300A0E7B0E08C9173
S123516083608C93000000000000000081E08093CC048093C8078093CE0480935D06EFE6D3
S1235180F0E080818D7F80838C918C7F8C93F901108215BC84E68093350608951F920F92E0
S12351A00FB60F9211240F900FBE0F901F901895813049F48093CC0486B590E090935406F0
S12351C0809353060895823021F481E08093C8070895833021F481E08093CE0408958430BC
S12351E019F481E080935D0608950F931F938091590490915A04845F914018F41092EF0791
S123520016C08091590490915A048D56974020F08EE08093EF070BC08091590490915A04CE
S123522064E670E00E946E2F65506093EF07E091EF07F0E0E151FE4F808180931301809104
S12352406C04882329F02091E3048091180109C0E0915D04F0915E04E153FB4F80812091A6
S12352601801829FC00111249093BA048093B9048091590490915A04825C914060F5809147
S123528000019091010182FF1CC08091B9049091BA042091190130911A01820F931F9093CF
S12352A0BA048093B90480919F079091A00784609093A00780939F0780911B018093B8047A
S12352C044C080919F079091A0078B7F9093A00780939F073AC080919F079091A0078B7F37
S12352E09093A00780939F078091B804823068F18091B80481508093B8042091B9043091B3
S1235300BA044091190150911A01E0911901F0911A0180911B017091B80460911B01240F93
S1235320351F90E0871B9109AC014E9FC0014F9F900D5E9F900D112470E00E946E2F261BE4
S1235340370B3093BA042093B90480916C04882309F0E8C08091F60787FD3FC08091F607AA
S12353608331DCF5E0915D04F0915E04E053FB4F4081E0915D04F0915E04E153FB4F2081DD
S12353800091B9041091BA043091CA078091F607E091180150E0421B510926EF8202C001F1
S12353A01124830F911D9C01429FC001439F900D529F900D11246AE070E00E94822FF0E036
S12353C06E9FC0016F9F900D7E9F900D1124800F911F9093BA048093B9048091CC0787FD09
S12353E03FC08091CC078F30DCF5E0915D04F0915E04ED51FB4F4081E0915D04F0915E0483
S1235400E153FB4F20810091B9041091BA043091F3078091CC07E091180150E0421B5109AC
S123542026EF8202C0011124830F911D9C01429FC001439F900D529F900D11246AE070E07E
S12354400E94822FF0E06E9FC0016F9F900D7E9F900D1124800F911F9093BA048093B904CD
S1235460809100019091010184FF5CC02091200430912104809100049091010428173907DF
S1235480FCF480910004909101042091200430912104821B930B64E070E00E94822F8091EF
S12354A05F04861710F460935F0480915F048A3018F089E080935F04809128018093BB046D
S12354C03091BB043430C8F08091B9049091BA04E0915F04F0E0EB51FE4F2081820F911D72
S12354E09093BA048093B90431503093BB0480919F079091A007806109C010925F04109224
S1235500BB0480919F079091A0078F7E9093A00780939F0780910004909101049093210436
S123552080932004809100019091010191FD09C08091F20386FF94C080916C04882309F49C
S12355408FC0809137068F5F809337069091370680913806981708F486C0109237068091DE
S1235560FC039091FD03E091CC07FF27E7FDF095EB5EF94F208130E02817390734F480913A
S1235580350690913606890F19C08091FC039091FD03E091CC07FF27E7FDF095EB5EF94F69
S12355A0208130E0821793075CF48091350618163CF48091350690913606891B809335066E
S12355C080919F079091A0079D7F9093A00780939F0720913506E091CC07FF27E7FDF095EA
S12355E0EB5EF94F8089332727FD309590E08C599F4F8217930754F4E091CC07FF27E7FDBE
S1235600F095EB5EF94F80898C591EC020913506E091CC07FF27E7FDF095EB5EF94F40898B
S1235620332727FD309584E690E0841B910928173907CCF4E091CC07FF27E7FDF095EB5EB5
S1235640F94F908984E6891B8093350680919F079091A00792609093A00780939F0703C0D2
S123566084E6809335068091B9049091BA048091C90780911E0120910A0430910B0490E0B1
S1235680C196821793070CF489C0809100019091010181FF83C080910A0490910B04C39792
S12356A0F4F0E0911C01F0911D0120911C0130911D0180910A0490910B0460911E0170E079
S12356C06E5C7F4FAC01429FC001439F900D529F900D11240E946E2FE61BF70B16C0809174
S12356E00A0490910B04889764F480911C0190911D0196958795FC01EE0FFF1FE80FF91F16
S123570004C0E0911C01F0911D018091B9049091BA0462E070E00E94822F70934C066093BA
S12357204B06CF019695879590934E0680934D068091B9049091BA04E80FF91FF093BA0423
S1235740E093B9048091B9049091BA0462E070E00E94822F7093500660934F0680911801B8
S123576090E09093520680935106309905C0809123019091240104C080911F019091200190
S1235780909322018093210180919F079091A00782609093A00780939F0711C080919F071E
S12357A09091A0078D7F9093A00780939F0780911F0190912001909322018093210180918F
S12357C010069091110683FF1CC0E091B904F091BA0420913D018091B9049091BA0464E1CB
S12357E070E00E94822F30E0629FC001639F900D729F900D11248E0F9F1F9093BA0480935F
S1235800B904809100019091010190FF4DC08091F4039091F503823891050CF045C0809173
S1235820B9049091BA0420912A01820F911D9093BA048093B904E091F403F091F50360912A
S1235840180120912A0182E890E08E1B9F0B70E0AB01849FB001859F700D949F700D1124CC
S12358608FEF90E0AB01489FB001499F700D589F700D1124882777FD8095982F30E040E0B5
S123588050E00E94432F20E43FE140E050E00E94952FC9012091B9043091BA04280F391FA0
S12358A03093BA042093B9042091B9043091BA048091180145EF849FC0011124821793075C
S12358C054F480911801849FC00111249093BA048093B9040BC08091B9049091BA041816E2
S12358E0190624F01092BA041092B9048091B9049091BA0490936104809360048091600491
S1235900909161049093A3078093A20778941F910F9108951F920F920FB60F9211242F93CC
S12359203F934F935F936F937F938F939F93AF93BF93EF93FF931092B100E091BF04F0E056
S12359402091A2073091A30786B59091C104891B280F311DEE0FFF1FE15CF94F318320833D
S123596086B580930F068091BF04813019F40E94F5280AC08091BF04823031F08091BF042A
S1235980833011F08091BF04FF91EF91BF91AF919F918F917F916F915F914F913F912F911B
S12359A00F900FBE0F901F9018951F93682F8FEF8093CD048091C1046093C10441E050E0F2
S12359C0162F181BACE0BEEF71E0FA01EE0FFF1FE15CF94F80819181181619066CF41093C3
S12359E0A107208131818091A10790E080959095820F931F91838083FA01EE0FFF1FE15C98
S1235A00F94F808191811816190624F180819181855D9E4FFCF0413049F44093CC0486B56B
S1235A2090E090935406809353060CC0423019F47093C80707C0433019F47093CE0402C00E
S1235A4070935D06FA01EE0FFF1FE15CF94FB183A08311C08091CD04FA01EE0FFF1FE15CE4
S1235A60F94F2081318190E02817390724F4808191818093CD044F5F5F4F4530510509F069
S1235A80A4CF8091CD048F3F21F08091CD04860F87BD1F9108951F920F920FB60F921124D9
S1235AA02F933F934F935F936F937F938F939F93AF93BF93EF93FF9386B50E94D52CFF91FC
S1235AC0EF91BF91AF919F918F917F916F915F914F913F912F910F900FBE0F901F9018958B
S1235AE01F920F920FB60F9211242F933F934F935F936F937F938F939F93AF93BF93EF93CF
S1235B00FF9386B50E94D52CFF91EF91BF91AF919F918F917F916F915F914F913F912F91B1
S1235B200F900FBE0F901F901895549A559A5C9A5D9A15BCEEE6F0E080818360808384E070
S1235B4085BD16BC82E187BD089511B88FEF84B915B887B98AB9089588E98093C100109291
S1235B60C50083E18093C40083E598E0909311088093100890930D0880930C0883E198E09F
S1235B8090930F0880930E0890939408809393081092120810923E0608951F920F920FB6DB
S1235BA00F9211248F939F93EF93FF9380911208882311F1E0911008F09111088191809383
S1235BC0C600F0931108E0931008E359F84030F083E598E0909311088093100880911208CE
S1235BE081508093120880911208882329F48091C1008F7D8093C100FF91EF919F918F919E
S1235C000F900FBE0F901F9018951F920F920FB60F9211242F938F939F93EF93FF938091F1
S1235C20C600E0919308F0919408808380913E068F5F80933E0680919308909194080196D4
S1235C4090939408809393088355984030F083E198E09093940880939308FF91EF919F917A
S1235C608F912F910F900FBE0F901F90189580913E06882319F42FEF3FEF1AC0F894809109
S1235C803E06815080933E06E0910E08F0910F082191F0930F08E0930E08E355F84030F010
S1235CA083E198E090930F0880930E08789430E0C9010895982F809112088F33E0F7809182
S1235CC01208803410F080E00895F894809112088F5F80931208E0910C08F0910D089083F5
S1235CE080910C0890910D08019690930D0880930C088359984030F083E598E090930D0863
S1235D0080930C088091C10080628093C100789481E00895CF93DF93EC0104C00E945A2E17
S1235D208111219688818823C9F781E0DF91CF9108958EED93E00E948A2E089586EE93E008
S1235D400E948A2E089580913E0608959F92AF92BF92CF92DF92EF92FF920F931F93DF93E9
S1235D60CF93CDB7DEB729970FB6F894DEBF0FBECDBF7C01062FDE011196E9EEF3E089E052
S1235D8001900D928150E1F719E099E0A92EB12C6E010894C11CD11C8CE2982E002371F073
S1235DA09501211B3109802F90E02817390730F01150F601E10FF11D908200E01150F60175
S1235DC0E10FF11DC7016AE070E00E946E2F805D8083C7016AE070E00E946E2F7B016115AD
S1235DE0710511F4002311F00630C0F219E0141B7E010894E11CF11C07C0F701E10FF11D0E
S1235E0080810E945A2E1F5F1930B8F329960FB6F894DEBF0FBECDBFCF91DF911F910F91BB
S1235E20FF90EF90DF90CF90BF90AF909F900895DF92EF92FF920F931F937B018C01FB014C
S1235E400995D82EC8010196F7010995982F8D2D1F910F91FF90EF90DF900895DF92EF92C7
S1235E60FF920F931F93D72E7A018C01FA010995C80101966D2DF70109951F910F91FF9024
S1235E80EF90DF900895629FD001739FF001829FE00DF11D649FE00DF11D929FF00D839F34
S1235EA0F00D749FF00D659FF00D9927729FB00DE11DF91F639FB00DE11DF91FBD01CF01C9
S1235EC011240895991B79E004C0991F961708F0961B881F7A95C9F780950895AA1BBB1B4A
S1235EE051E107C0AA1FBB1FA617B70710F0A61BB70B881F991F5A95A9F780959095BC011F
S1235F00CD01089597FB092E07260AD077FD04D0E5DF06D000201AF4709561957F4F0895CC
S1235F20F6F7909581959F4F0895A1E21A2EAA1BBB1BFD010DC0AA1FBB1FEE1FFF1FA217F2
S1235F40B307E407F50720F0A21BB30BE40BF50B661F771F881F991F1A9469F760957095A0
S1235F60809590959B01AC01BD01CF01089597FB092E05260ED057FD04D0D7DF0AD0001CC9
S1235F8038F450954095309521953F4F4F4F5F4F0895F6F790958095709561957F4F8F4F57
S1235FA09F4F0895F894FFCF2F00010002000300040005000600070008003228E8039001CF
S1235FC00614001E1E003C581B581B88136419121E01010203040A0411C4098813C409643A
S1235FE000DCE64003020A1432469628000000000000000000000000000000000000000042
S123600000000000000000000000000000000000000000000000000000000000000000007C
S1236020000000000000000000000000000102030405060708090A0B0C0D0E0F10010203CE
S12360400405060708090A0B0C0D0E0F100102030405060708090A0B0C0D0E0F10141617F1
S123606018191A1B1C1D1E1F2021222324191A1B1C1D1E1F2021222324252627271E1F2032
S123608022232425262728292A2B2C2D2E000204060708090A0C0E28262422201E1E1E1E80
S12360A01E1E1E1E1E1E1EF0FF80BBE0880465484BA438022BF0207019CC13860F440CC254
S12360C009D0074C061B052A046A03D1025602F201A1015F012801FB00D600B7009D0087DA
S12360E0007500660059004D0044003C0034002E0029002500F0FF80BBE0880465484BA4B9
S123610038022BF0207019CC13860F440CC209D0074C061B052A046A03D1025602F201A14B
S1236120015F012801FB00D600B7009D0087007500660059004D0044003C0034002E002999
S1236140002500F0FF80BBE0880465484BA438022BF0207019CC13860F440CC209D0074C34
S1236160061B052A046A03D1025602F201A1015F012801FB00D600B7009D0087007500668A
S12361800059004D0044003C0034002E0029002500F0FF80BBE0880465484BA438022BF09E
S12361A0207019CC13860F440CC209D0074C061B052A046A03D1025602F201A1015F012877
S12361C001FB00D600B7009D0087007500660059004D0044003C0034002E0029002500005D
S12361E000F5047E05AE066C08C00AB30D630F8B10D7118813000000000A000F001E003C6A
S1236200007800FA007201E00180028002000008000A000C000E00C80A4A067E048403ACAD
S12362200D641A002000270032003E0066008E00B202EB02240337034B03560361037003A4
S1236240E800D600C200B0009D008A00780078006500520040002D001900070000000100AE
S1236260010001175A5A5A505050505050505050505050500A0004010402030000030000C8
S11D6280FA32040404041B5B481B5B324A000D0A00202020202020202020DD
S5030315E4
